:10000000A0C0F3C1B8C0B7C0B6C0B5C0B4C0B3C01B
:10001000B2C0B1C0B0C0AFC0AEC0ADC0ACC0ABC06C
:10002000AAC0A9C0A8C016032800530029004E008A
:10003000450053005F0075007300620018037200F2
:100040006100700068006E00650074002E006E0094
:100050006500740004030904090222000101008004
:100060003209040000010300000009210101000120
:100070002200000705810308000A0A033600300049
:100080003100310005010905A1010901A100093074
:100090000931150026FF00750895028102C0050987
:1000A0001901290815002501750195088102C01262
:1000B000010101000000088117970A0301010203F2
:1000C0000105010902A1010901A100050919012980
:1000D00002150025019502750181029501750681C1
:1000E000030501093009311581257F7508950281C5
:1000F00006C0C012010101000000088117990A031F
:10010000010102030105010905A1010901A100097D
:10011000300931150026FF00750895028102C005DF
:10012000091901290415002501750195048102C0F2
:1001300012010101000000088117960A0301010263
:10014000030111241FBECFE5D4E0DEBFCDBF10E018
:10015000A0E6B0E0E6EAF0E102C005900D92A03A18
:10016000B107D9F710E0A0EAB0E001C01D92AE3FA0
:10017000B107E1F759C344CFCF93DC01C62F6930F3
:1001800008F0C8E02BE49091B80090FD23EC80913A
:10019000620087FF04C09F5F9093B80003C08FEF99
:1001A000809362002093E700E8EEF0E02C2F2150CE
:1001B0002F3F19F08D918193FACF6C2F88EE90E04C
:1001C000C6D2CC5FC0936200CF9108951F93CF93A6
:1001D0009091F700992309F48CC0935097FD87C044
:1001E000E0EAF0E0E091E600EF5F40E0C0E88091F7
:1001F000F4008D3209F077C0983009F074C0808126
:10020000807609F06DC021EE30E04093E1008181FD
:10021000882321F44093E20042E057C0853021F466
:1002200082818093F80051C08630D9F5C0EC83817B
:10023000813039F44091F9002091E4003091E500DB
:1002400044C0823021F442E228E530E03EC08330F1
:10025000C9F48281882321F444E024E530E035C0EC
:10026000813021F448E12CE330E02FC0823021F4CA
:1002700046E126E230E029C0833039F54AE02AE73A
:1002800030E023C0813221F449E02AE630E01DC08D
:100290008232D9F44091E3002091FC003091FD00BE
:1002A00014C0883021F441E02BEF30E00EC08930DB
:1002B00021F482818093FB0008C08A3011F441E070
:1002C00004C08B3011F44093B8003093F6002093B3
:1002D000F5008781882339F48681841720F402C0D1
:1002E000CF0139D2482FC093B600409364001092DA
:1002F000F700909164009F3F09F44FC08091630024
:1003000087FF4BC0692F993008F068E0961B9093E7
:1003100064001BE48091B60080FD13EC8F5F809336
:10032000B600A9EDB0E0E091F500F091F600962F4F
:10033000915086FF13C09F3FB9F084919D012F5FBC
:100340003F4FAF014F5F5F4F9150E157F04011F4C5
:100350008091E3008C93D901FA01EDCF9F3F21F00A
:1003600081918D939150FACFF093F600E093F500D0
:100370007727C62F693040F489ED90E0E8D19C2FB3
:100380009C5FC83030F402C01EE192E08FEF809392
:1003900064001093D8009093630080B3857019F0C7
:1003A0001092B70011C08091B700882369F494E6D9
:1003B00080B3857049F49150D9F781E08093B700FC
:1003C0009093F8009093F300CF911F91089580EAE5
:1003D00090E08093F2000B968093E60085B78360EF
:1003E00085BF8BB780648BBF08950F930FB70F93B2
:1003F000809BFECF809B06C0809B04C0809B02C078
:10040000000000C01F933F932F9331E014E000B32E
:10041000102710FD32E0102F3A95C9F700FDE7C014
:1004200000B3102717952FE72795DF9310B3012707
:1004300007952795CF93C091F20000B31027179529
:1004400027953BE0D0E04F9310B301270795279500
:100450004FEF000055C0809BFECF809B06C0809B65
:1004600004C0809B02C0000000C0DF9100C0CDCF5F
:1004700010B3157079F1407C2C6F13C000B3057078
:1004800049F141782C6F15C0057021F1102F2C6FA8
:1004900000B319C000B30570E9F04E7F2C6F18C08F
:1004A00038F300B30570B1F0102717952795243065
:1004B00028F310B3012707952795422749934FEF5B
:1004C00000B3243008F3102717952795243010F334
:1004D00010B31570E1F10127079527952430F0F04E
:1004E00000B30570A1F11027179527952430E0F08F
:1004F00010B30127079527953A9541F12430D0F0A4
:1005000000B3057021F11027179527952430C0F00E
:1005100010B30127079527952430C2CF10B315706B
:10052000B1F04C7F2C6FDCCF00B3057081F0487FB9
:100530002C6FDECF10B3157051F0407F2C6FE0CFE1
:1005400000B3057021F0407E2C6FE2CF3DC03C2F00
:10055000C091F2003C1B00E433300ABFA8F10881CF
:100560001981412F1F772091F3000D3289F1013E4F
:1005700079F10936C1F00777033431F51091FA00AB
:10058000112311F10091F7000030D1F53430DAF188
:100590003093F7001093F4000091E600C093E6005A
:1005A0000093F20030C0121779F447FD3AC0309141
:1005B00063003F3F29F10FEF00936300C8EDD0E0E7
:1005C00025C000270093FA004F91CF91DF910FC013
:1005D0001217B9F70093FA000FEF0093640000932D
:1005E00063004F91CF910AB706FD35CFDF9100E44C
:1005F0000ABF2F913F911F910F910FBF0F91189537
:10060000C0E6D0E002C0C1E6D0E032E05F9302B3C2
:100610000A7F016002BB55E011B3156011BB20E8F1
:1006200019C0309162003F3F59F30FEF0093620011
:10063000C7EED0E0EBCF052710E002BB10C00527C6
:1006400010E0089402BB13C0052710E015C0052771
:1006500010E019C020FF052702BB279517951C3F06
:1006600050F720FF0527279502BB17951C3F38F749
:1006700020FF05272795179502BB1C3F28F720FF71
:100680000527279517951C3F02BB08F700C0499125
:1006900020FF052702BB279517951C3F80F520FFFB
:1006A0000527279502BB17951C3F68F520FF0527F6
:1006B0002795179502BB1C3F58F520FF0527279566
:1006C00017951C3F02BB38F5242F3A9519F60A7F7F
:1006D0005F9102BB32E03A95F1F71091F800C256F3
:1006E000D04011F01093F300016011B31A7F02BBE8
:1006F0000A7F4F91CF9111BB02BBDF9178CF0527C5
:1007000010E002BBCACF052710E0089402BBCDCF92
:10071000052710E0CFCF052710E0D3CFA82FB92FA2
:100720008FEF9FEF41E050EA615070F02D9138E07B
:10073000722F782796958795269570FF02C084279B
:1007400095273A95A9F7F0CF809590950895E6DF23
:100750008D939D930895FC012BEB30E03093F600D0
:100760002093F5008081992780769070809719F505
:100770008181813081F4E091B900F091BA00008864
:10078000F189E02DC9010995E091B900F091BA0015
:10079000808199270895823049F481EC90E090930C
:1007A000F6008093F50081E090E008958A3019F416
:1007B00083818093C10080E090E00895EF92FF92E2
:1007C0000F931F93CF93DF93AC01415050408FEFB5
:1007D0004F3F580711F180E3E82E85E7F82E012DF1
:1007E000112D23E130E0C7010197F1F7215030408E
:1007F00037FFF9CFA0E3B5E7C0E0D0E021E330E078
:10080000CD010197F1F72150304037FFF9CF41502A
:1008100050408FEF4F3F580721F7DF91CF911F9145
:100820000F91FF90EF900895CFE5D4E0DEBFCDBFEC
:10083000C0E001E01C2FB89A87B3897F87BB88B3DB
:10084000866088BBC09880E395E70197F1F786B38F
:10085000992786709070002E02C0959587950A940E
:10086000E2F78230910531F0039761F081E090E08A
:10087000A5DFFCCFF9D39093BA008093B90081E053
:1008800090E014C051D1FC019093BA008093B9005C
:100890000284F385E02D0995E8D1882329F068D3F7
:1008A0009093BA008093B90082E090E087DFE091F6
:1008B000B900F091BA00848195819093FD008093F6
:1008C000FC0082818093E30080859185009731F060
:1008D0009093E5008093E400868107C080E391E077
:1008E0009093E5008093E400CED38093F90014BA8E
:1008F0008FEF85BB98EF92BB95E091BB90E0915054
:10090000F1F78150D9F781BB85E083BF8FE085BDCA
:1009100084EC83BDE091B900F091BA000284F385C4
:10092000E02D099554DD7894A89550DC002349F01A
:10093000E091B900F091BA000484F585E02D0995A5
:1009400000E008B600FE0CC091E098BF8091C100A5
:10095000882331F0153010F0155002C0182FC92F20
:1009600008B607FE18C080E888BFCC23A1F4E09148
:10097000B900F091BA000484F585E02D0995E09165
:10098000B900F091BA000684F785E02D0995882317
:1009900059F2C1E002C0CC2339F2809162008F3F4E
:1009A00019F6C0E0E091B900F091BA000088F18931
:1009B000E02D8BEB90E00995E091B900F091BA0041
:1009C00060818BEB90E0D8DBAFCF90E0AC9A80E316
:1009D0008A95F1F7AC9828E130E040E050E067E01C
:1009E00070E0822F8A95F1F7AD98990F9B9B9160EB
:1009F000822F8A95F1F7AD9A6150704077FFF1CF61
:100A00009093C20028E130E040E050E067E070E001
:100A1000822F8A95F1F7AD9896959B9B9068822FCF
:100A20008A95F1F7AD9A6150704077FFF1CF9093BE
:100A3000C30008951F931FB7F894A49AA59AA3988A
:100A4000AB9AAD9AAC98C1DF1FBF1F9108958091FA
:100A5000770090917800892B39F0109278001092ED
:100A6000770021E030E00BC042E050E064EC70E041
:100A700082EC90E00BD3282F332727FD3095C90156
:100A80000895CF93DC01892B09F444C08091C20002
:100A9000C091C30060E870E0FB01482F552740FF7C
:100AA00002C0EFEFF0E041FF02C0E0E0F0E042FF03
:100AB00002C06FEF70E043FF02C060E070E0EC93B3
:100AC000FD0161839A01220F232F221F330B3195E1
:100AD000CA0180749070A5E095958795AA95E1F775
:100AE000282BCA018072907073E0959587957A954E
:100AF000E1F7282B4071507055954795242B8C2F8A
:100B000099278F70907034E0880F991F3A95E1F71C
:100B1000282B22838091C2009091C3009093C5003E
:100B20008093C400CF91089584E890E090936A0088
:100B30008093690085E690E00895FC01AC9A80E31B
:100B40008A95F1F7AC9828E130E040E050E097E07A
:100B5000822F8A95F1F7AD98822F8A95F1F7AD9A99
:100B6000915097FFF5CF28E130E040E050E097E06A
:100B7000822F8A95F1F7AD988081880F80839B99A9
:100B800002C081608083822F8A95F1F7AD9A9150DF
:100B900097FFEECF0895AF92BF92CF92DF92EF9280
:100BA000FF920F931F93CF93DF93CDB7DEB72197BB
:100BB0000FB6F894DEBF0FBECDBF46E0C42ED12CD9
:100BC00033E0A32EB12CA822B922CE010196B5DFC5
:100BD000898199278073907024E0959587952A954F
:100BE000E1F78A159B0529F4B092CB00A092CA00C8
:100BF0002BC088EB9BE00197F1F724E030E040E068
:100C000050E080E3E82EF12C012D112D6EE170E013
:100C1000AC9A822F8A95F1F7AD98AD9A822F8A957A
:100C2000F1F7AC988E2D8A95F1F76150704077FFFF
:100C3000EFCF80E89BEB0197F1F70894C108D1084A
:100C4000C114D10409F0C1CF21960FB6F894DEBFCC
:100C50000FBECDBFDF91CF911F910F91FF90EF900D
:100C6000DF90CF90BF90AF900895CF93DF93CDB733
:100C7000DEB721970FB6F894DEBF0FBECDBFCE0111
:100C800001965BDF898199278F7090708130910583
:100C900011F080E090E021960FB6F894DEBF0FBE11
:100CA000CDBFDF91CF9108950F931F93CF93DF9323
:100CB000CDB7DEB721970FB6F894DEBF0FBECDBF1C
:100CC00010E0012FCE01019638DF8981282F3327CC
:100CD000C9018F709070019761F54091CC005091DF
:100CE000CD004115510551F5C90166E096958795EE
:100CF0006A95E1F78130910591F0823091051CF4FD
:100D0000892B49F00DC08230910521F0039741F401
:100D1000CA0105C040DF8091CA009091CB003BDF43
:100D2000CE0101960ADF898199278F709070019713
:100D300029F01092CD001092CC0059C081E090E0D3
:100D40009093CD008093CC0089818093D00080E780
:100D500097E10197F1F780E08A95F1F740E250E0E2
:100D600060E070E027E030E0842F8A95F1F7AD98DD
:100D7000110F9B9B11600000AD9A2150304037FF4E
:100D8000F3CF40E250E060E070E027E030E0842FF5
:100D90008A95F1F7AD98000F9B9B01600000AD9A1A
:100DA0002150304037FFF3CF202F2F77412F4F773F
:100DB00007FD219517FD4195332727FD309580913B
:100DC000C8009091C900820F931F9093C90080932F
:100DD000C800242F332727FD30958091C6009091BD
:100DE000C700820F931F9093C7008093C60021967F
:100DF0000FB6F894DEBF0FBECDBFDF91CF911F912C
:100E00000F910895A49AA59AA398AB9AAD9AAC981D
:100E10004BDF8091D000992776E0969587957A955B
:100E2000E1F78130910569F0823091051CF4892B3E
:100E300031F008958230910531F0039729F480E074
:100E400090E0A9DE0895A7DE089540918B005091AF
:100E50008C004115510529F010928C0010928B00E6
:100E60001CC09091D0008091D1009817B1F42091CE
:100E7000C8003091C9008091D2009091D30028170A
:100E8000390759F42091C6003091C7008091D400F1
:100E90009091D5002817390719F081E090E0089566
:100EA000CA010895FC01892B09F461C08091CE002C
:100EB0009091CF00892B41F0108211821282109202
:100EC000CF001092CE0008958091D0009927A6E01F
:100ED00096958795AA95E1F780838091C8009091B7
:100EE000C9002FEF8138920714F421E807C0803839
:100EF000910514F02FE702C02091C8008091C60030
:100F00009091C7003FEF8138930714F441E807C080
:100F10008038910514F04FE702C04091C60021834C
:100F20004283332727FD30953093D3002093D2009E
:100F3000552747FD50955093D5004093D40080919C
:100F4000D0008093D1008091C8009091C900821B8D
:100F5000930B9093C9008093C8008091C600909134
:100F6000C700841B950B9093C7008093C60008951B
:100F700081EC90E090937E0080937D008FEA90E07A
:100F8000909382008093810089E790E00895A49A6D
:100F9000A59AA398AB9AAD9AAC98089590E0AC9AB4
:100FA00080E38A95F1F7AC9828E130E040E050E02A
:100FB00067E070E0822F8A95F1F7AD98990F9B9BBF
:100FC0009160822F8A95F1F7AD9A6150704077FF5A
:100FD000F1CF9093D60008958091D6009091D700DC
:100FE000891B992787FD90950895FC01892BB9F1FC
:100FF00020E830E0B9018091D600482F552740FF06
:1010000002C06FEF70E041FF02C060E070E042FF9D
:1010100002C02FEF30E043FF02C020E030E06083E9
:1010200021839A01220F232F221F330B3195CA01EE
:101030008074907065E0959587956A95E1F7282B07
:10104000CA018072907033E0959587953A95E1F7E3
:10105000282B4071507055954795242B2283809101
:10106000D6008093D700089585E091E09093920098
:101070008093910083EF90E0909396008093950089
:101080008DE890E0089582E190E00895FB01DC0195
:1010900004C08D910190801921F441505040C8F74F
:0610A000881B990B089566
:1010A6005AD2FFFFFF03002B000000000000001AC9
:1010B60005E5042705410501000300320000001282
:1010C6000000000207540625075207010003002B03
:1010D60000000012000000C707CE07EC07F5070066
:00000001FF
